 jsound

 Timestamp is ffffffff (Sun Feb  7 06:28:15 2106)

 Preferred load address is 10000000

 Start         Length     Name                   Class
 0001:00000000 00000030H .text$di                CODE
 0001:00000030 00006a6cH .text$mn                CODE
 0001:00006a9c 00000014H .text$yd                CODE
 0002:00000000 00000198H .idata$5                DATA
 0002:00000198 00000004H .00cfg                  DATA
 0002:0000019c 00000004H .CRT$XCA                DATA
 0002:000001a0 00000008H .CRT$XCU                DATA
 0002:000001a8 00000004H .CRT$XCZ                DATA
 0002:000001ac 00000004H .CRT$XIA                DATA
 0002:000001b0 00000004H .CRT$XIZ                DATA
 0002:000001b4 00000004H .CRT$XPA                DATA
 0002:000001b8 00000004H .CRT$XPZ                DATA
 0002:000001bc 00000004H .CRT$XTA                DATA
 0002:000001c0 00000010H .CRT$XTZ                DATA
 0002:000001c4 00000000H .gfids$y                DATA
 0002:000001d0 00000740H .rdata                  DATA
 0002:00000910 00000130H .rdata$r                DATA
 0002:00000a40 00000004H .rdata$sxdata           DATA
 0002:00000a44 000002e4H .rdata$zzzdbg           DATA
 0002:00000d28 00000004H .rtc$IAA                DATA
 0002:00000d2c 00000004H .rtc$IZZ                DATA
 0002:00000d30 00000004H .rtc$TAA                DATA
 0002:00000d34 00000004H .rtc$TZZ                DATA
 0002:00000d38 00000118H .xdata$x                DATA
 0002:00000e50 00000db4H .edata                  DATA
 0002:00001c04 000000dcH .idata$2                DATA
 0002:00001ce0 00000014H .idata$3                DATA
 0002:00001cf4 00000198H .idata$4                DATA
 0002:00001e8c 00000766H .idata$6                DATA
 0003:00000000 00000044H .data                   DATA
 0003:00000044 0000007cH .data$r                 DATA
 0003:000000c0 00000cfcH .bss                    DATA
 0004:00000000 00000060H .rsrc$01                DATA
 0004:00000060 00000310H .rsrc$02                DATA

  Address         Publics by Value              Rva+Base       Lib:Object

 0000:00000000       ___guard_fids_count        00000000     <absolute>
 0000:00000000       ___hybrid_code_map_count   00000000     <absolute>
 0000:00000000       ___hybrid_code_map         00000000     <absolute>
 0000:00000000       ___guard_longjmp_table     00000000     <absolute>
 0000:00000000       ___volatile_metadata       00000000     <absolute>
 0000:00000000       ___guard_iat_count         00000000     <absolute>
 0000:00000000       ___enclave_config          00000000     <absolute>
 0000:00000000       ___dynamic_value_reloc_table 00000000     <absolute>
 0000:00000000       ___guard_iat_table         00000000     <absolute>
 0000:00000000       ___guard_longjmp_count     00000000     <absolute>
 0000:00000000       ___guard_fids_table        00000000     <absolute>
 0000:00000000       ___hybrid_auxiliary_iat    00000000     <absolute>
 0000:00000001       ___safe_se_handler_count   00000001     <absolute>
 0000:00000100       ___guard_flags             00000100     <absolute>
 0000:00000000       ___ImageBase               10000000     <linker-defined>
 0001:00000030       _DAUDIO_AddAudioFormat     10001030 f   DirectAudioDevice.obj
 0001:00000096       _Java_com_sun_media_sound_DirectAudioDevice_nAvailable@20 10001096 f   DirectAudioDevice.obj
 0001:000000bc       _Java_com_sun_media_sound_DirectAudioDevice_nClose@20 100010bc f   DirectAudioDevice.obj
 0001:000000f5       _Java_com_sun_media_sound_DirectAudioDevice_nFlush@20 100010f5 f   DirectAudioDevice.obj
 0001:00000114       _Java_com_sun_media_sound_DirectAudioDevice_nGetBufferSize@20 10001114 f   DirectAudioDevice.obj
 0001:0000013a       _Java_com_sun_media_sound_DirectAudioDevice_nGetBytePosition@28 1000113a f   DirectAudioDevice.obj
 0001:00000164       _Java_com_sun_media_sound_DirectAudioDevice_nGetFormats@24 10001164 f   DirectAudioDevice.obj
 0001:000001b2       _Java_com_sun_media_sound_DirectAudioDevice_nIsStillDraining@20 100011b2 f   DirectAudioDevice.obj
 0001:000001d8       _Java_com_sun_media_sound_DirectAudioDevice_nOpen@52 100011d8 f   DirectAudioDevice.obj
 0001:00000285       _Java_com_sun_media_sound_DirectAudioDevice_nRead@32 10001285 f   DirectAudioDevice.obj
 0001:00000307       _Java_com_sun_media_sound_DirectAudioDevice_nRequiresServicing@20 10001307 f   DirectAudioDevice.obj
 0001:0000032c       _Java_com_sun_media_sound_DirectAudioDevice_nService@20 1000132c f   DirectAudioDevice.obj
 0001:0000034b       _Java_com_sun_media_sound_DirectAudioDevice_nSetBytePosition@28 1000134b f   DirectAudioDevice.obj
 0001:00000373       _Java_com_sun_media_sound_DirectAudioDevice_nStart@20 10001373 f   DirectAudioDevice.obj
 0001:00000392       _Java_com_sun_media_sound_DirectAudioDevice_nStop@20 10001392 f   DirectAudioDevice.obj
 0001:000003b1       _Java_com_sun_media_sound_DirectAudioDevice_nWrite@40 100013b1 f   DirectAudioDevice.obj
 0001:0000061f       _handleGainAndConversion   1000161f f   DirectAudioDevice.obj
 0001:00001643       _handleSignEndianConversion 10002643 f   DirectAudioDevice.obj
 0001:0000172b       _Java_com_sun_media_sound_DirectAudioDeviceProvider_nGetNumDevices@8 1000272b f   DirectAudioDeviceProvider.obj
 0001:00001733       _Java_com_sun_media_sound_DirectAudioDeviceProvider_nNewDirectAudioDeviceInfo@12 10002733 f   DirectAudioDeviceProvider.obj
 0001:00001846       _getDirectAudioDeviceDescription 10002846 f   DirectAudioDeviceProvider.obj
 0001:000018a5       _Java_com_sun_media_sound_MidiInDevice_nClose@16 100028a5 f   MidiInDevice.obj
 0001:000018b2       _Java_com_sun_media_sound_MidiInDevice_nGetMessages@16 100028b2 f   MidiInDevice.obj
 0001:00001a90       _Java_com_sun_media_sound_MidiInDevice_nGetTimeStamp@16 10002a90 f   MidiInDevice.obj
 0001:00001a90       _Java_com_sun_media_sound_MidiOutDevice_nGetTimeStamp@16 10002a90 f   MidiOutDevice.obj
 0001:00001aae       _Java_com_sun_media_sound_MidiInDevice_nOpen@12 10002aae f   MidiInDevice.obj
 0001:00001af5       _Java_com_sun_media_sound_MidiInDevice_nStart@16 10002af5 f   MidiInDevice.obj
 0001:00001b1e       _Java_com_sun_media_sound_MidiInDevice_nStop@16 10002b1e f   MidiInDevice.obj
 0001:00001b2b       _Java_com_sun_media_sound_MidiInDeviceProvider_nGetDescription@12 10002b2b f   MidiInDeviceProvider.obj
 0001:00001b9b       _Java_com_sun_media_sound_MidiInDeviceProvider_nGetName@12 10002b9b f   MidiInDeviceProvider.obj
 0001:00001c0b       _Java_com_sun_media_sound_MidiInDeviceProvider_nGetNumDevices@8 10002c0b f   MidiInDeviceProvider.obj
 0001:00001c13       _Java_com_sun_media_sound_MidiOutDeviceProvider_nGetVendor@12 10002c13 f   MidiOutDeviceProvider.obj
 0001:00001c13       _Java_com_sun_media_sound_MidiInDeviceProvider_nGetVendor@12 10002c13 f   MidiInDeviceProvider.obj
 0001:00001c83       _Java_com_sun_media_sound_MidiInDeviceProvider_nGetVersion@12 10002c83 f   MidiInDeviceProvider.obj
 0001:00001cf3       _Java_com_sun_media_sound_MidiOutDevice_nClose@16 10002cf3 f   MidiOutDevice.obj
 0001:00001d00       _Java_com_sun_media_sound_MidiOutDevice_nOpen@12 10002d00 f   MidiOutDevice.obj
 0001:00001d3e       _Java_com_sun_media_sound_MidiOutDevice_nSendLongMessage@32 10002d3e f   MidiOutDevice.obj
 0001:00001d92       _Java_com_sun_media_sound_MidiOutDevice_nSendShortMessage@28 10002d92 f   MidiOutDevice.obj
 0001:00001da9       _Java_com_sun_media_sound_MidiOutDeviceProvider_nGetDescription@12 10002da9 f   MidiOutDeviceProvider.obj
 0001:00001e19       _Java_com_sun_media_sound_MidiOutDeviceProvider_nGetName@12 10002e19 f   MidiOutDeviceProvider.obj
 0001:00001e89       _Java_com_sun_media_sound_MidiOutDeviceProvider_nGetNumDevices@8 10002e89 f   MidiOutDeviceProvider.obj
 0001:00001e91       _Java_com_sun_media_sound_MidiOutDeviceProvider_nGetVersion@12 10002e91 f   MidiOutDeviceProvider.obj
 0001:00001f01       _UnicodeToUTF8             10002f01 f   PLATFORM_API_WinOS_Charset_Util.obj
 0001:00001f4d       _UnicodeToUTF8AndCopy      10002f4d f   PLATFORM_API_WinOS_Charset_Util.obj
 0001:00001f81       ??0Data@DS_StartBufferHelper@@QAE@XZ 10002f81 f   PLATFORM_API_WinOS_DirectSound.obj
 0001:00001fd0       ??1Data@DS_StartBufferHelper@@QAE@XZ 10002fd0 f   PLATFORM_API_WinOS_DirectSound.obj
 0001:00002006       ?DS_CheckUnderrun@@YAXPAUDS_Info@@KK@Z 10003006 f   PLATFORM_API_WinOS_DirectSound.obj
 0001:0000203a       ?DS_GetAvailable@@YAHPAUDS_Info@@PAK1PAHH@Z 1000303a f   PLATFORM_API_WinOS_DirectSound.obj
 0001:0000217d       ?DS_GetDescEnum@@YGHPAU_GUID@@PBG1PAUtag_DirectAudioDeviceDescription@@@Z 1000317d f   PLATFORM_API_WinOS_DirectSound.obj
 0001:000021c0       ?DS_RefreshCacheEnum@@YGHPAU_GUID@@PBD1PAUDS_RefreshCacheStruct@@@Z 100031c0 f   PLATFORM_API_WinOS_DirectSound.obj
 0001:00002247       ?DS_addDeviceRef@@YAHH@Z   10003247 f   PLATFORM_API_WinOS_DirectSound.obj
 0001:000022f5       ?DS_addPos@@YAHPAUDS_Info@@HH@Z 100032f5 f i PLATFORM_API_WinOS_DirectSound.obj
 0001:0000230f       ?DS_clearBuffer@@YAXPAUDS_Info@@H@Z 1000330f f   PLATFORM_API_WinOS_DirectSound.obj
 0001:000024be       ?DS_createSoundBuffer@@YAPAXPAUDS_Info@@MHHH@Z 100034be f   PLATFORM_API_WinOS_DirectSound.obj
 0001:000025aa       ?DS_destroySoundBuffer@@YAXPAUDS_Info@@@Z 100035aa f   PLATFORM_API_WinOS_DirectSound.obj
 0001:000025d3       ?DS_removeDeviceRef@@YAXH@Z 100035d3 f   PLATFORM_API_WinOS_DirectSound.obj
 0001:0000260b       ?StartBuffer@DS_StartBufferHelper@@SAJPAUDS_Info@@@Z 1000360b f   PLATFORM_API_WinOS_DirectSound.obj
 0001:0000265e       ?ThreadProc@DS_StartBufferHelper@@KGKPAX@Z 1000365e f   PLATFORM_API_WinOS_DirectSound.obj
 0001:000026c0       ?createWaveFormat@@YAXPAUWAVEFORMATEXTENSIBLE@@HHHH@Z 100036c0 f   PLATFORM_API_WinOS_DirectSound.obj
 0001:0000276b       ?estimatePositionFromAvail@@YA_JPAUDS_Info@@_JHH@Z 1000376b f   PLATFORM_API_WinOS_DirectSound.obj
 0001:00002795       ?findCacheItemByGUID@@YAHPAU_GUID@@H@Z 10003795 f   PLATFORM_API_WinOS_DirectSound.obj
 0001:000027d9       ?findCacheItemByMixerIndex@@YAHH@Z 100037d9 f   PLATFORM_API_WinOS_DirectSound.obj
 0001:00002800       ?isEqualGUID@@YAHPAU_GUID@@0@Z 10003800 f   PLATFORM_API_WinOS_DirectSound.obj
 0001:0000283a       _DAUDIO_Close              1000383a f   PLATFORM_API_WinOS_DirectSound.obj
 0001:0000285c       _DAUDIO_Flush              1000385c f   PLATFORM_API_WinOS_DirectSound.obj
 0001:000028ac       _DAUDIO_GetAvailable       100038ac f   PLATFORM_API_WinOS_DirectSound.obj
 0001:000028cd       _DAUDIO_GetBufferSize      100038cd f   PLATFORM_API_WinOS_DirectSound.obj
 0001:000028d5       _DAUDIO_GetBytePosition    100038d5 f   PLATFORM_API_WinOS_DirectSound.obj
 0001:00002908       _DAUDIO_GetDirectAudioDeviceCount 10003908 f   PLATFORM_API_WinOS_DirectSound.obj
 0001:00002a37       _DAUDIO_GetDirectAudioDeviceDescription 10003a37 f   PLATFORM_API_WinOS_DirectSound.obj
 0001:00002acd       _DAUDIO_GetFormats         10003acd f   PLATFORM_API_WinOS_DirectSound.obj
 0001:00002b59       _DAUDIO_Open               10003b59 f   PLATFORM_API_WinOS_DirectSound.obj
 0001:00002c7b       _DAUDIO_Read               10003c7b f   PLATFORM_API_WinOS_DirectSound.obj
 0001:00002d82       _DAUDIO_RequiresServicing  10003d82 f   PLATFORM_API_WinOS_DirectSound.obj
 0001:00002d8c       _DAUDIO_Service            10003d8c f   PLATFORM_API_WinOS_DirectSound.obj
 0001:00002dcc       _DAUDIO_SetBytePosition    10003dcc f   PLATFORM_API_WinOS_DirectSound.obj
 0001:00002dcc       @_guard_check_icall_nop@4  10003dcc f   MSVCRT:guard_support.obj
 0001:00002dcd       _DAUDIO_Start              10003dcd f   PLATFORM_API_WinOS_DirectSound.obj
 0001:00002e5d       _DAUDIO_StillDraining      10003e5d f   PLATFORM_API_WinOS_DirectSound.obj
 0001:00002e92       _DAUDIO_Stop               10003e92 f   PLATFORM_API_WinOS_DirectSound.obj
 0001:00002eb8       _DAUDIO_Write              10003eb8 f   PLATFORM_API_WinOS_DirectSound.obj
 0001:0000302d       ??0Data@MidiIn_OpenHelper@@QAE@XZ 1000402d f   PLATFORM_API_WinOS_MidiIn.obj
 0001:00003079       ??1Data@MidiIn_OpenHelper@@QAE@XZ 10004079 f   PLATFORM_API_WinOS_MidiIn.obj
 0001:000030af       ?MIDI_IN_PutMessage@@YGXPAUHMIDIIN__@@IIII@Z 100040af f   PLATFORM_API_WinOS_MidiIn.obj
 0001:0000315e       ?ThreadProc@MidiIn_OpenHelper@@KGKPAX@Z 1000415e f   PLATFORM_API_WinOS_MidiIn.obj
 0001:000031a8       ?getMidiInCaps@@YAHHPAUtagMIDIINCAPSW@@PAH@Z 100041a8 f   PLATFORM_API_WinOS_MidiIn.obj
 0001:000031c8       ?midiInOpen@MidiIn_OpenHelper@@SAIHPAUtag_MidiDeviceHandle@@@Z 100041c8 f   PLATFORM_API_WinOS_MidiIn.obj
 0001:00003222       ?prepareBuffers@@YAHPAUtag_MidiDeviceHandle@@@Z 10004222 f   PLATFORM_API_WinOS_MidiIn.obj
 0001:0000326e       ?unprepareBuffers@@YAHPAUtag_MidiDeviceHandle@@@Z 1000426e f   PLATFORM_API_WinOS_MidiIn.obj
 0001:000032af       _MIDI_IN_CloseDevice       100042af f   PLATFORM_API_WinOS_MidiIn.obj
 0001:00003302       _MIDI_IN_GetDeviceVendor   10004302 f   PLATFORM_API_WinOS_MidiIn.obj
 0001:00003302       _MIDI_OUT_GetDeviceVendor  10004302 f   PLATFORM_API_WinOS_MidiOut.obj
 0001:00003302       _MIDI_IN_GetDeviceDescription 10004302 f   PLATFORM_API_WinOS_MidiIn.obj
 0001:00003308       _MIDI_IN_GetDeviceName     10004308 f   PLATFORM_API_WinOS_MidiIn.obj
 0001:00003364       _MIDI_IN_GetDeviceVersion  10004364 f   PLATFORM_API_WinOS_MidiIn.obj
 0001:000033d9       _MIDI_IN_GetErrorStr       100043d9 f   PLATFORM_API_WinOS_MidiIn.obj
 0001:000033fa       _MIDI_IN_GetMessage        100043fa f   PLATFORM_API_WinOS_MidiIn.obj
 0001:0000343f       _MIDI_IN_GetNumDevices     1000443f f   PLATFORM_API_WinOS_MidiIn.obj
 0001:00003445       _MIDI_OUT_GetTimeStamp     10004445 f   PLATFORM_API_WinOS_MidiOut.obj
 0001:00003445       _MIDI_IN_GetTimeStamp      10004445 f   PLATFORM_API_WinOS_MidiIn.obj
 0001:0000344a       _MIDI_IN_OpenDevice        1000444a f   PLATFORM_API_WinOS_MidiIn.obj
 0001:00003512       _MIDI_IN_ReleaseMessage    10004512 f   PLATFORM_API_WinOS_MidiIn.obj
 0001:0000355c       _MIDI_IN_StartDevice       1000455c f   PLATFORM_API_WinOS_MidiIn.obj
 0001:000035af       _MIDI_IN_StopDevice        100045af f   PLATFORM_API_WinOS_MidiIn.obj
 0001:000035fb       ___local_stdio_printf_options 100045fb f i PLATFORM_API_WinOS_MidiIn.obj
 0001:00003601       __vsnprintf_l              10004601 f i PLATFORM_API_WinOS_MidiIn.obj
 0001:00003634       _sprintf                   10004634 f i PLATFORM_API_WinOS_MidiIn.obj
 0001:0000364e       _MIDI_OUT_CloseDevice      1000464e f   PLATFORM_API_WinOS_MidiOut.obj
 0001:000036dd       _MIDI_OUT_GetDeviceDescription 100046dd f   PLATFORM_API_WinOS_MidiOut.obj
 0001:00003794       _MIDI_OUT_GetDeviceName    10004794 f   PLATFORM_API_WinOS_MidiOut.obj
 0001:000037f0       _MIDI_OUT_GetDeviceVersion 100047f0 f   PLATFORM_API_WinOS_MidiOut.obj
 0001:0000385e       _MIDI_OUT_GetErrorStr      1000485e f   PLATFORM_API_WinOS_MidiOut.obj
 0001:0000387f       _MIDI_OUT_GetNumDevices    1000487f f   PLATFORM_API_WinOS_MidiOut.obj
 0001:00003887       _MIDI_OUT_OpenDevice       10004887 f   PLATFORM_API_WinOS_MidiOut.obj
 0001:0000396c       _MIDI_OUT_SendLongMessage  1000496c f   PLATFORM_API_WinOS_MidiOut.obj
 0001:00003aae       _MIDI_OUT_SendShortMessage 10004aae f   PLATFORM_API_WinOS_MidiOut.obj
 0001:00003ac9       _freeLongBuffer            10004ac9 f   PLATFORM_API_WinOS_MidiOut.obj
 0001:00003b24       _freeLongBuffers           10004b24 f   PLATFORM_API_WinOS_MidiOut.obj
 0001:00003b63       _getMidiOutCaps            10004b63 f   PLATFORM_API_WinOS_MidiOut.obj
 0001:00003b8e       _unprepareLongBuffers      10004b8e f   PLATFORM_API_WinOS_MidiOut.obj
 0001:00003bd5       _PORT_Close                10004bd5 f   PLATFORM_API_WinOS_Ports.obj
 0001:00003c44       _PORT_GetControls          10004c44 f   PLATFORM_API_WinOS_Ports.obj
 0001:00003e4c       _PORT_GetFloatValue        10004e4c f   PLATFORM_API_WinOS_Ports.obj
 0001:00003ee7       _PORT_GetIntValue          10004ee7 f   PLATFORM_API_WinOS_Ports.obj
 0001:00003f2b       _PORT_GetPortCount         10004f2b f   PLATFORM_API_WinOS_Ports.obj
 0001:00003f3c       _PORT_GetPortMixerCount    10004f3c f   PLATFORM_API_WinOS_Ports.obj
 0001:00003f42       _PORT_GetPortMixerDescription 10004f42 f   PLATFORM_API_WinOS_Ports.obj
 0001:00003fc5       _PORT_GetPortName          10004fc5 f   PLATFORM_API_WinOS_Ports.obj
 0001:00004011       _PORT_GetPortType          10005011 f   PLATFORM_API_WinOS_Ports.obj
 0001:00004044       _PORT_Open                 10005044 f   PLATFORM_API_WinOS_Ports.obj
 0001:00004310       _PORT_SetFloatValue        10005310 f   PLATFORM_API_WinOS_Ports.obj
 0001:000043cf       _PORT_SetIntValue          100053cf f   PLATFORM_API_WinOS_Ports.obj
 0001:00004449       _addAllControls            10005449 f   PLATFORM_API_WinOS_Ports.obj
 0001:00004476       _addCompoundControl        10005476 f   PLATFORM_API_WinOS_Ports.obj
 0001:000044a7       _componentType2type        100054a7 f   PLATFORM_API_WinOS_Ports.obj
 0001:0000450e       _createLineControls        1000550e f   PLATFORM_API_WinOS_Ports.obj
 0001:0000461f       _createMuxControl          1000561f f   PLATFORM_API_WinOS_Ports.obj
 0001:0000481b       _createPortControl         1000581b f   PLATFORM_API_WinOS_Ports.obj
 0001:000049a6       _findDestLine              100059a6 f   PLATFORM_API_WinOS_Ports.obj
 0001:000049ce       _getControlCount           100059ce f   PLATFORM_API_WinOS_Ports.obj
 0001:00004a79       _getControlInfo            10005a79 f   PLATFORM_API_WinOS_Ports.obj
 0001:00004aee       _getControlValue           10005aee f   PLATFORM_API_WinOS_Ports.obj
 0001:00004b0b       _getDestinationCount       10005b0b f   PLATFORM_API_WinOS_Ports.obj
 0001:00004b43       _getFakeBalance            10005b43 f   PLATFORM_API_WinOS_Ports.obj
 0001:00004bcd       _getFakeVolume             10005bcd f   PLATFORM_API_WinOS_Ports.obj
 0001:00004c13       _getMixerLineByDestination 10005c13 f   PLATFORM_API_WinOS_Ports.obj
 0001:00004c48       _getMixerLineBySource      10005c48 f   PLATFORM_API_WinOS_Ports.obj
 0001:00004c84       _lineHasControls           10005c84 f   PLATFORM_API_WinOS_Ports.obj
 0001:00004cfc       _setControlValue           10005cfc f   PLATFORM_API_WinOS_Ports.obj
 0001:00004d19       _setFakeVolume             10005d19 f   PLATFORM_API_WinOS_Ports.obj
 0001:00004da6       _MIDI_CreateLock           10005da6 f   PLATFORM_API_WinOS_Util.obj
 0001:00004dbd       _MIDI_DestroyLock          10005dbd f   PLATFORM_API_WinOS_Util.obj
 0001:00004dd5       _MIDI_GetTimeStamp         10005dd5 f   PLATFORM_API_WinOS_Util.obj
 0001:00004e1b       _MIDI_Lock                 10005e1b f   PLATFORM_API_WinOS_Util.obj
 0001:00004e2d       _MIDI_SetStartTime         10005e2d f   PLATFORM_API_WinOS_Util.obj
 0001:00004e45       _MIDI_Unlock               10005e45 f   PLATFORM_API_WinOS_Util.obj
 0001:00004e57       _MIDI_WinCreateEmptyLongBufferQueue 10005e57 f   PLATFORM_API_WinOS_Util.obj
 0001:00004e6c       _MIDI_WinCreateLongBufferQueue 10005e6c f   PLATFORM_API_WinOS_Util.obj
 0001:00004efd       _MIDI_WinDestroyLongBufferQueue 10005efd f   PLATFORM_API_WinOS_Util.obj
 0001:00004f2d       _Java_com_sun_media_sound_Platform_nIsBigEndian@8 10005f2d f   Platform.obj
 0001:00004f35       _GetInternalErrorStr       10005f35 f   PlatformMidi.obj
 0001:00004f7e       _MIDI_CreateQueue          10005f7e f   PlatformMidi.obj
 0001:00004fb5       _MIDI_DestroyQueue         10005fb5 f   PlatformMidi.obj
 0001:00004fe3       _MIDI_IN_InternalGetErrorString 10005fe3 f   PlatformMidi.obj
 0001:0000500a       _MIDI_OUT_InternalGetErrorString 1000600a f   PlatformMidi.obj
 0001:00005031       _MIDI_QueueAddLong         10006031 f   PlatformMidi.obj
 0001:000050e0       _MIDI_QueueAddShort        100060e0 f   PlatformMidi.obj
 0001:0000516a       _MIDI_QueueClear           1000616a f   PlatformMidi.obj
 0001:00005190       _MIDI_QueueRead            10006190 f   PlatformMidi.obj
 0001:000051c8       _MIDI_QueueRemove          100061c8 f   PlatformMidi.obj
 0001:00005215       _Java_com_sun_media_sound_PortMixer_nClose@16 10006215 f   PortMixer.obj
 0001:0000522c       _Java_com_sun_media_sound_PortMixer_nControlGetFloatValue@16 1000622c f   PortMixer.obj
 0001:0000524f       _Java_com_sun_media_sound_PortMixer_nControlGetIntValue@16 1000624f f   PortMixer.obj
 0001:0000526c       _Java_com_sun_media_sound_PortMixer_nControlSetFloatValue@20 1000626c f   PortMixer.obj
 0001:00005290       _Java_com_sun_media_sound_PortMixer_nControlSetIntValue@20 10006290 f   PortMixer.obj
 0001:000052ac       _Java_com_sun_media_sound_PortMixer_nGetControls@24 100062ac f   PortMixer.obj
 0001:00005332       _Java_com_sun_media_sound_PortMixer_nGetPortCount@16 10006332 f   PortMixer.obj
 0001:0000534f       _Java_com_sun_media_sound_PortMixer_nGetPortName@20 1000634f f   PortMixer.obj
 0001:000053ac       _Java_com_sun_media_sound_PortMixer_nGetPortType@20 100063ac f   PortMixer.obj
 0001:000053ce       _Java_com_sun_media_sound_PortMixer_nOpen@12 100063ce f   PortMixer.obj
 0001:000053dc       _PORT_AddControl           100063dc f   PortMixer.obj
 0001:00005408       _PORT_NewBooleanControl    10006408 f   PortMixer.obj
 0001:000054a3       _PORT_NewCompoundControl   100064a3 f   PortMixer.obj
 0001:0000557a       _PORT_NewFloatControl      1000657a f   PortMixer.obj
 0001:000056b1       _Java_com_sun_media_sound_PortMixerProvider_nGetNumDevices@8 100066b1 f   PortMixerProvider.obj
 0001:000056b9       _Java_com_sun_media_sound_PortMixerProvider_nNewPortMixerInfo@12 100066b9 f   PortMixerProvider.obj
 0001:000057c0       _getPortMixerDescription   100067c0 f   PortMixerProvider.obj
 0001:00005815       _ThrowJavaMessageException 10006815 f   Utilities.obj
 0001:00005835       _UTIL_IsBigEndianPlatform  10006835 f   Utilities.obj
 0001:00005835       ___scrt_stub_for_is_c_termination_complete 10006835 f   MSVCRT:ucrt_stubs.obj
 0001:00005835       __is_c_termination_complete 10006835 f   MSVCRT:ucrt_stubs.obj
 0001:00005838       _DirectSoundCreate@12      10006838 f   dsound:DSOUND.dll
 0001:0000583e       _DirectSoundEnumerateA@8   1000683e f   dsound:DSOUND.dll
 0001:00005844       _DirectSoundEnumerateW@8   10006844 f   dsound:DSOUND.dll
 0001:0000584a       _DirectSoundCaptureCreate@12 1000684a f   dsound:DSOUND.dll
 0001:00005850       _DirectSoundCaptureEnumerateA@8 10006850 f   dsound:DSOUND.dll
 0001:00005856       _DirectSoundCaptureEnumerateW@8 10006856 f   dsound:DSOUND.dll
 0001:0000585c       @__security_check_cookie@4 1000685c f   MSVCRT:secchk.obj
 0001:0000586d       ??_U@YAPAXI@Z              1000686d f   MSVCRT:new_array.obj
 0001:00005876       ??_V@YAXPAX@Z              10006876 f   MSVCRT:delete_array.obj
 0001:000058bf       ___scrt_acquire_startup_lock 100068bf f   MSVCRT:utility.obj
 0001:000058f1       ___scrt_dllmain_after_initialize_c 100068f1 f   MSVCRT:utility.obj
 0001:0000591c       ___scrt_dllmain_before_initialize_c 1000691c f   MSVCRT:utility.obj
 0001:0000592a       ___scrt_dllmain_crt_thread_attach 1000692a f   MSVCRT:utility.obj
 0001:00005949       ___scrt_dllmain_crt_thread_detach 10006949 f   MSVCRT:utility.obj
 0001:00005956       ___scrt_dllmain_exception_filter 10006956 f   MSVCRT:utility.obj
 0001:0000598a       ___scrt_dllmain_uninitialize_c 1000698a f   MSVCRT:utility.obj
 0001:000059ad       ___scrt_dllmain_uninitialize_critical 100069ad f   MSVCRT:utility.obj
 0001:000059ba       ___scrt_initialize_crt     100069ba f   MSVCRT:utility.obj
 0001:000059f3       ___scrt_initialize_onexit_tables 100069f3 f   MSVCRT:utility.obj
 0001:00005a98       ___scrt_is_nonwritable_in_current_image 10006a98 f   MSVCRT:utility.obj
 0001:00005b2c       ___scrt_release_startup_lock 10006b2c f   MSVCRT:utility.obj
 0001:00005b49       ___scrt_uninitialize_crt   10006b49 f   MSVCRT:utility.obj
 0001:00005b71       __onexit                   10006b71 f   MSVCRT:utility.obj
 0001:00005bac       _atexit                    10006bac f   MSVCRT:utility.obj
 0001:00005bd0       __ftoui3                   10006bd0 f   MSVCRT:ftol3.obj
 0001:00005bdf       __ftoul3                   10006bdf f   MSVCRT:ftol3.obj
 0001:00005bee       __ftol3                    10006bee f   MSVCRT:ftol3.obj
 0001:00005bfb       __ftol3_NaN                10006bfb f   MSVCRT:ftol3.obj
 0001:00005c13       __ftol3_work               10006c13 f   MSVCRT:ftol3.obj
 0001:00005c99       __ftol3_common             10006c99 f   MSVCRT:ftol3.obj
 0001:00005d5b       __ftol3_arg_error          10006d5b f   MSVCRT:ftol3.obj
 0001:00005d6d       __ftol3_except             10006d6d f   MSVCRT:ftol3.obj
 0001:00005db1       __dtoui3                   10006db1 f   MSVCRT:ftol3.obj
 0001:00005dc0       __dtoul3                   10006dc0 f   MSVCRT:ftol3.obj
 0001:00005dcf       __dtol3                    10006dcf f   MSVCRT:ftol3.obj
 0001:00005ddc       __dtol3_NaN                10006ddc f   MSVCRT:ftol3.obj
 0001:00005df9       __dtol3_work               10006df9 f   MSVCRT:ftol3.obj
 0001:00005ee0       __ultod3                   10006ee0 f   MSVCRT:ftol3.obj
 0001:00005f20       __ltod3                    10006f20 f   MSVCRT:ftol3.obj
 0001:00005f50       __allmul                   10006f50 f   MSVCRT:llmul.obj
 0001:000062a4       __DllMainCRTStartup@12     100072a4 f   MSVCRT:dll_dllmain.obj
 0001:000062c7       ___raise_securityfailure   100072c7 f   MSVCRT:gs_report.obj
 0001:000062ef       ___report_gsfailure        100072ef f   MSVCRT:gs_report.obj
 0001:000063e8       ??2@YAPAXI@Z               100073e8 f   MSVCRT:new_scalar.obj
 0001:00006418       ??3@YAXPAX@Z               10007418 f   MSVCRT:delete_scalar.obj
 0001:0000641d       ___isa_available_init      1000741d f   MSVCRT:cpu_disp.obj
 0001:000065b4       __get_startup_argv_mode    100075b4 f   MSVCRT:argv_mode.obj
 0001:000065b8       ___scrt_is_ucrt_dll_in_use 100075b8 f   MSVCRT:ucrt_detection.obj
 0001:000065c4       ___scrt_fastfail           100075c4 f   MSVCRT:utility_desktop.obj
 0001:000066de       __crt_debugger_hook        100076de f   MSVCRT:utility_desktop.obj
 0001:000066f0       __SEH_prolog4              100076f0 f   MSVCRT:sehprolg4.obj
 0001:00006736       __SEH_epilog4              10007736 f   MSVCRT:sehprolg4.obj
 0001:0000674b       __except_handler4          1000774b f   MSVCRT:chandler4gs.obj
 0001:000067bb       ___security_init_cookie    100077bb f   MSVCRT:gs_support.obj
 0001:00006806       _DllMain@12                10007806 f   MSVCRT:dll_dllmain_stub.obj
 0001:00006828       ?__scrt_initialize_type_info@@YAXXZ 10007828 f   MSVCRT:tncleanup.obj
 0001:00006834       ?__scrt_uninitialize_type_info@@YAXXZ 10007834 f   MSVCRT:tncleanup.obj
 0001:00006840       ___local_stdio_scanf_options 10007840 f i MSVCRT:default_local_stdio_options.obj
 0001:00006846       ___scrt_initialize_default_local_stdio_options 10007846 f   MSVCRT:default_local_stdio_options.obj
 0001:00006863       ___scrt_get_dyn_tls_init_callback 10007863 f   MSVCRT:dyn_tls_init.obj
 0001:00006869       __RTC_Initialize           10007869 f   MSVCRT:initsect.obj
 0001:00006895       __RTC_Terminate            10007895 f   MSVCRT:initsect.obj
 0001:000068c1       ??0bad_alloc@std@@QAE@ABV01@@Z 100078c1 f i MSVCRT:throw_bad_alloc.obj
 0001:000068dc       ??0bad_alloc@std@@QAE@XZ   100078dc f i MSVCRT:throw_bad_alloc.obj
 0001:000068f4       ??0bad_array_new_length@std@@QAE@ABV01@@Z 100078f4 f i MSVCRT:throw_bad_alloc.obj
 0001:0000690f       ??0bad_array_new_length@std@@QAE@XZ 1000790f f i MSVCRT:throw_bad_alloc.obj
 0001:00006927       ??0exception@std@@QAE@ABV01@@Z 10007927 f i MSVCRT:throw_bad_alloc.obj
 0001:00006953       ??1bad_alloc@std@@UAE@XZ   10007953 f i MSVCRT:throw_bad_alloc.obj
 0001:00006953       ??1bad_array_new_length@std@@UAE@XZ 10007953 f i MSVCRT:throw_bad_alloc.obj
 0001:00006964       ??_Gexception@std@@UAEPAXI@Z 10007964 f i MSVCRT:throw_bad_alloc.obj
 0001:00006964       ??_Eexception@std@@UAEPAXI@Z 10007964 f i MSVCRT:throw_bad_alloc.obj
 0001:00006964       ??_Ebad_array_new_length@std@@UAEPAXI@Z 10007964 f i MSVCRT:throw_bad_alloc.obj
 0001:00006964       ??_Ebad_alloc@std@@UAEPAXI@Z 10007964 f i MSVCRT:throw_bad_alloc.obj
 0001:00006964       ??_Gbad_alloc@std@@UAEPAXI@Z 10007964 f i MSVCRT:throw_bad_alloc.obj
 0001:00006964       ??_Gbad_array_new_length@std@@UAEPAXI@Z 10007964 f i MSVCRT:throw_bad_alloc.obj
 0001:00006991       ?__scrt_throw_std_bad_alloc@@YAXXZ 10007991 f   MSVCRT:throw_bad_alloc.obj
 0001:000069ae       ?__scrt_throw_std_bad_array_new_length@@YAXXZ 100079ae f   MSVCRT:throw_bad_alloc.obj
 0001:000069cb       ?what@exception@std@@UBEPBDXZ 100079cb f i MSVCRT:throw_bad_alloc.obj
 0001:000069d8       ??3@YAXPAXI@Z              100079d8 f   MSVCRT:delete_scalar_size.obj
 0001:000069e6       ??_Gtype_info@@UAEPAXI@Z   100079e6 f i MSVCRT:std_type_info_static.obj
 0001:000069e6       ??_Etype_info@@UAEPAXI@Z   100079e6 f i MSVCRT:std_type_info_static.obj
 0001:00006a09       _IsProcessorFeaturePresent@4 10007a09 f   kernel32:KERNEL32.dll
 0001:00006a0f       _memcpy                    10007a0f f   vcruntime:VCRUNTIME140.dll
 0001:00006a15       _memset                    10007a15 f   vcruntime:VCRUNTIME140.dll
 0001:00006a1b       _memcmp                    10007a1b f   vcruntime:VCRUNTIME140.dll
 0001:00006a21       __except_handler4_common   10007a21 f   vcruntime:VCRUNTIME140.dll
 0001:00006a27       ___std_type_info_destroy_list 10007a27 f   vcruntime:VCRUNTIME140.dll
 0001:00006a2d       ___std_exception_copy      10007a2d f   vcruntime:VCRUNTIME140.dll
 0001:00006a33       ___std_exception_destroy   10007a33 f   vcruntime:VCRUNTIME140.dll
 0001:00006a39       __CxxThrowException@8      10007a39 f   vcruntime:VCRUNTIME140.dll
 0001:00006a3f       _free                      10007a3f f   ucrt:api-ms-win-crt-heap-l1-1-0.dll
 0001:00006a45       _malloc                    10007a45 f   ucrt:api-ms-win-crt-heap-l1-1-0.dll
 0001:00006a4b       _strcpy                    10007a4b f   ucrt:api-ms-win-crt-string-l1-1-0.dll
 0001:00006a51       __seh_filter_dll           10007a51 f   ucrt:api-ms-win-crt-runtime-l1-1-0.dll
 0001:00006a57       __configure_narrow_argv    10007a57 f   ucrt:api-ms-win-crt-runtime-l1-1-0.dll
 0001:00006a5d       __initialize_narrow_environment 10007a5d f   ucrt:api-ms-win-crt-runtime-l1-1-0.dll
 0001:00006a63       __initialize_onexit_table  10007a63 f   ucrt:api-ms-win-crt-runtime-l1-1-0.dll
 0001:00006a69       __register_onexit_function 10007a69 f   ucrt:api-ms-win-crt-runtime-l1-1-0.dll
 0001:00006a6f       __execute_onexit_table     10007a6f f   ucrt:api-ms-win-crt-runtime-l1-1-0.dll
 0001:00006a75       __crt_atexit               10007a75 f   ucrt:api-ms-win-crt-runtime-l1-1-0.dll
 0001:00006a7b       __cexit                    10007a7b f   ucrt:api-ms-win-crt-runtime-l1-1-0.dll
 0001:00006a81       __except1                  10007a81 f   ucrt:api-ms-win-crt-math-l1-1-0.dll
 0001:00006a87       __initterm                 10007a87 f   ucrt:api-ms-win-crt-runtime-l1-1-0.dll
 0001:00006a8d       __initterm_e               10007a8d f   ucrt:api-ms-win-crt-runtime-l1-1-0.dll
 0001:00006a93       __callnewh                 10007a93 f   ucrt:api-ms-win-crt-heap-l1-1-0.dll
 0001:00006a99       ___acrt_thread_detach      10007a99 f   MSVCRT:ucrt_stubs.obj
 0001:00006a99       ___acrt_initialize         10007a99 f   MSVCRT:ucrt_stubs.obj
 0001:00006a99       ___vcrt_initialize         10007a99 f   MSVCRT:ucrt_stubs.obj
 0001:00006a99       ___acrt_uninitialize       10007a99 f   MSVCRT:ucrt_stubs.obj
 0001:00006a99       ___scrt_stub_for_acrt_uninitialize 10007a99 f   MSVCRT:ucrt_stubs.obj
 0001:00006a99       ___scrt_stub_for_acrt_uninitialize_critical 10007a99 f   MSVCRT:ucrt_stubs.obj
 0001:00006a99       ___vcrt_thread_attach      10007a99 f   MSVCRT:ucrt_stubs.obj
 0001:00006a99       ___scrt_stub_for_acrt_thread_attach 10007a99 f   MSVCRT:ucrt_stubs.obj
 0001:00006a99       ___vcrt_uninitialize       10007a99 f   MSVCRT:ucrt_stubs.obj
 0001:00006a99       ___vcrt_thread_detach      10007a99 f   MSVCRT:ucrt_stubs.obj
 0001:00006a99       ___scrt_stub_for_acrt_initialize 10007a99 f   MSVCRT:ucrt_stubs.obj
 0001:00006a99       ___vcrt_uninitialize_critical 10007a99 f   MSVCRT:ucrt_stubs.obj
 0001:00006a99       ___acrt_thread_attach      10007a99 f   MSVCRT:ucrt_stubs.obj
 0001:00006a99       ___acrt_uninitialize_critical 10007a99 f   MSVCRT:ucrt_stubs.obj
 0001:00006a99       ___scrt_stub_for_acrt_thread_detach 10007a99 f   MSVCRT:ucrt_stubs.obj
 0002:00000000       __imp__DirectSoundEnumerateA@8 10008000     dsound:DSOUND.dll
 0002:00000004       __imp__DirectSoundEnumerateW@8 10008004     dsound:DSOUND.dll
 0002:00000008       __imp__DirectSoundCaptureCreate@12 10008008     dsound:DSOUND.dll
 0002:0000000c       __imp__DirectSoundCaptureEnumerateA@8 1000800c     dsound:DSOUND.dll
 0002:00000010       __imp__DirectSoundCaptureEnumerateW@8 10008010     dsound:DSOUND.dll
 0002:00000014       __imp__DirectSoundCreate@12 10008014     dsound:DSOUND.dll
 0002:00000018       \177DSOUND_NULL_THUNK_DATA 10008018     dsound:DSOUND.dll
 0002:0000001c       __imp__InitializeSListHead@4 1000801c     kernel32:KERNEL32.dll
 0002:00000020       __imp__DisableThreadLibraryCalls@4 10008020     kernel32:KERNEL32.dll
 0002:00000024       __imp__GetSystemTimeAsFileTime@4 10008024     kernel32:KERNEL32.dll
 0002:00000028       __imp__GetCurrentThreadId@0 10008028     kernel32:KERNEL32.dll
 0002:0000002c       __imp__GetCurrentProcessId@0 1000802c     kernel32:KERNEL32.dll
 0002:00000030       __imp__QueryPerformanceCounter@4 10008030     kernel32:KERNEL32.dll
 0002:00000034       __imp__IsDebuggerPresent@0 10008034     kernel32:KERNEL32.dll
 0002:00000038       __imp__IsProcessorFeaturePresent@4 10008038     kernel32:KERNEL32.dll
 0002:0000003c       __imp__TerminateProcess@8  1000803c     kernel32:KERNEL32.dll
 0002:00000040       __imp__GetCurrentProcess@0 10008040     kernel32:KERNEL32.dll
 0002:00000044       __imp__SetUnhandledExceptionFilter@4 10008044     kernel32:KERNEL32.dll
 0002:00000048       __imp__UnhandledExceptionFilter@4 10008048     kernel32:KERNEL32.dll
 0002:0000004c       __imp__DeleteCriticalSection@4 1000804c     kernel32:KERNEL32.dll
 0002:00000050       __imp__Sleep@4             10008050     kernel32:KERNEL32.dll
 0002:00000054       __imp__CreateThread@24     10008054     kernel32:KERNEL32.dll
 0002:00000058       __imp__CreateEventA@16     10008058     kernel32:KERNEL32.dll
 0002:0000005c       __imp__WaitForSingleObject@8 1000805c     kernel32:KERNEL32.dll
 0002:00000060       __imp__SetEvent@4          10008060     kernel32:KERNEL32.dll
 0002:00000064       __imp__LeaveCriticalSection@4 10008064     kernel32:KERNEL32.dll
 0002:00000068       __imp__EnterCriticalSection@4 10008068     kernel32:KERNEL32.dll
 0002:0000006c       __imp__InitializeCriticalSection@4 1000806c     kernel32:KERNEL32.dll
 0002:00000070       __imp__CloseHandle@4       10008070     kernel32:KERNEL32.dll
 0002:00000074       __imp__WideCharToMultiByte@32 10008074     kernel32:KERNEL32.dll
 0002:00000078       \177KERNEL32_NULL_THUNK_DATA 10008078     kernel32:KERNEL32.dll
 0002:0000007c       __imp__GetForegroundWindow@0 1000807c     user32:USER32.dll
 0002:00000080       __imp__GetDesktopWindow@0  10008080     user32:USER32.dll
 0002:00000084       \177USER32_NULL_THUNK_DATA 10008084     user32:USER32.dll
 0002:00000088       __imp__memcpy              10008088     vcruntime:VCRUNTIME140.dll
 0002:0000008c       __imp____std_exception_copy 1000808c     vcruntime:VCRUNTIME140.dll
 0002:00000090       __imp____std_exception_destroy 10008090     vcruntime:VCRUNTIME140.dll
 0002:00000094       __imp__memset              10008094     vcruntime:VCRUNTIME140.dll
 0002:00000098       __imp____std_type_info_destroy_list 10008098     vcruntime:VCRUNTIME140.dll
 0002:0000009c       __imp__memcmp              1000809c     vcruntime:VCRUNTIME140.dll
 0002:000000a0       __imp___except_handler4_common 100080a0     vcruntime:VCRUNTIME140.dll
 0002:000000a4       __imp___CxxThrowException@8 100080a4     vcruntime:VCRUNTIME140.dll
 0002:000000a8       \177VCRUNTIME140_NULL_THUNK_DATA 100080a8     vcruntime:VCRUNTIME140.dll
 0002:000000ac       __imp__mixerSetControlDetails@12 100080ac     winmm:WINMM.dll
 0002:000000b0       __imp__mixerGetControlDetailsA@12 100080b0     winmm:WINMM.dll
 0002:000000b4       __imp__mixerGetNumDevs@0   100080b4     winmm:WINMM.dll
 0002:000000b8       __imp__timeEndPeriod@4     100080b8     winmm:WINMM.dll
 0002:000000bc       __imp__timeBeginPeriod@4   100080bc     winmm:WINMM.dll
 0002:000000c0       __imp__midiOutReset@4      100080c0     winmm:WINMM.dll
 0002:000000c4       __imp__midiOutLongMsg@12   100080c4     winmm:WINMM.dll
 0002:000000c8       __imp__midiOutShortMsg@8   100080c8     winmm:WINMM.dll
 0002:000000cc       __imp__midiOutUnprepareHeader@12 100080cc     winmm:WINMM.dll
 0002:000000d0       __imp__mixerGetLineControlsA@12 100080d0     winmm:WINMM.dll
 0002:000000d4       __imp__midiOutClose@4      100080d4     winmm:WINMM.dll
 0002:000000d8       __imp__midiOutOpen@20      100080d8     winmm:WINMM.dll
 0002:000000dc       __imp__midiOutGetErrorTextA@12 100080dc     winmm:WINMM.dll
 0002:000000e0       __imp__midiOutGetDevCapsW@12 100080e0     winmm:WINMM.dll
 0002:000000e4       __imp__midiOutGetNumDevs@0 100080e4     winmm:WINMM.dll
 0002:000000e8       __imp__midiInReset@4       100080e8     winmm:WINMM.dll
 0002:000000ec       __imp__midiInStop@4        100080ec     winmm:WINMM.dll
 0002:000000f0       __imp__midiInStart@4       100080f0     winmm:WINMM.dll
 0002:000000f4       __imp__midiInAddBuffer@12  100080f4     winmm:WINMM.dll
 0002:000000f8       __imp__midiInUnprepareHeader@12 100080f8     winmm:WINMM.dll
 0002:000000fc       __imp__midiInPrepareHeader@12 100080fc     winmm:WINMM.dll
 0002:00000100       __imp__midiInClose@4       10008100     winmm:WINMM.dll
 0002:00000104       __imp__midiInOpen@20       10008104     winmm:WINMM.dll
 0002:00000108       __imp__midiInGetErrorTextA@12 10008108     winmm:WINMM.dll
 0002:0000010c       __imp__midiInGetDevCapsW@12 1000810c     winmm:WINMM.dll
 0002:00000110       __imp__midiInGetNumDevs@0  10008110     winmm:WINMM.dll
 0002:00000114       __imp__timeGetTime@0       10008114     winmm:WINMM.dll
 0002:00000118       __imp__mixerGetLineInfoA@12 10008118     winmm:WINMM.dll
 0002:0000011c       __imp__mixerClose@4        1000811c     winmm:WINMM.dll
 0002:00000120       __imp__mixerOpen@20        10008120     winmm:WINMM.dll
 0002:00000124       __imp__midiOutPrepareHeader@12 10008124     winmm:WINMM.dll
 0002:00000128       __imp__mixerGetDevCapsW@12 10008128     winmm:WINMM.dll
 0002:0000012c       \177WINMM_NULL_THUNK_DATA  1000812c     winmm:WINMM.dll
 0002:00000130       __imp__malloc              10008130     ucrt:api-ms-win-crt-heap-l1-1-0.dll
 0002:00000134       __imp___callnewh           10008134     ucrt:api-ms-win-crt-heap-l1-1-0.dll
 0002:00000138       __imp__free                10008138     ucrt:api-ms-win-crt-heap-l1-1-0.dll
 0002:0000013c       \177api-ms-win-crt-heap-l1-1-0_NULL_THUNK_DATA 1000813c     ucrt:api-ms-win-crt-heap-l1-1-0.dll
 0002:00000140       __imp___except1            10008140     ucrt:api-ms-win-crt-math-l1-1-0.dll
 0002:00000144       \177api-ms-win-crt-math-l1-1-0_NULL_THUNK_DATA 10008144     ucrt:api-ms-win-crt-math-l1-1-0.dll
 0002:00000148       __imp___initterm           10008148     ucrt:api-ms-win-crt-runtime-l1-1-0.dll
 0002:0000014c       __imp___initterm_e         1000814c     ucrt:api-ms-win-crt-runtime-l1-1-0.dll
 0002:00000150       __imp___seh_filter_dll     10008150     ucrt:api-ms-win-crt-runtime-l1-1-0.dll
 0002:00000154       __imp___configure_narrow_argv 10008154     ucrt:api-ms-win-crt-runtime-l1-1-0.dll
 0002:00000158       __imp___initialize_narrow_environment 10008158     ucrt:api-ms-win-crt-runtime-l1-1-0.dll
 0002:0000015c       __imp___initialize_onexit_table 1000815c     ucrt:api-ms-win-crt-runtime-l1-1-0.dll
 0002:00000160       __imp___register_onexit_function 10008160     ucrt:api-ms-win-crt-runtime-l1-1-0.dll
 0002:00000164       __imp___execute_onexit_table 10008164     ucrt:api-ms-win-crt-runtime-l1-1-0.dll
 0002:00000168       __imp___crt_atexit         10008168     ucrt:api-ms-win-crt-runtime-l1-1-0.dll
 0002:0000016c       __imp___cexit              1000816c     ucrt:api-ms-win-crt-runtime-l1-1-0.dll
 0002:00000170       \177api-ms-win-crt-runtime-l1-1-0_NULL_THUNK_DATA 10008170     ucrt:api-ms-win-crt-runtime-l1-1-0.dll
 0002:00000174       __imp____stdio_common_vsprintf 10008174     ucrt:api-ms-win-crt-stdio-l1-1-0.dll
 0002:00000178       \177api-ms-win-crt-stdio-l1-1-0_NULL_THUNK_DATA 10008178     ucrt:api-ms-win-crt-stdio-l1-1-0.dll
 0002:0000017c       __imp__strncpy             1000817c     ucrt:api-ms-win-crt-string-l1-1-0.dll
 0002:00000180       __imp__strcpy              10008180     ucrt:api-ms-win-crt-string-l1-1-0.dll
 0002:00000184       \177api-ms-win-crt-string-l1-1-0_NULL_THUNK_DATA 10008184     ucrt:api-ms-win-crt-string-l1-1-0.dll
 0002:00000188       __imp__CoInitialize@4      10008188     ole32:ole32.dll
 0002:0000018c       __imp__CoInitializeEx@8    1000818c     ole32:ole32.dll
 0002:00000190       __imp__CoUninitialize@0    10008190     ole32:ole32.dll
 0002:00000194       \177ole32_NULL_THUNK_DATA  10008194     ole32:ole32.dll
 0002:00000198       ___guard_check_icall_fptr  10008198     MSVCRT:guard_support.obj
 0002:0000019c       ___xc_a                    1000819c     MSVCRT:initializers.obj
 0002:000001a8       ___xc_z                    100081a8     MSVCRT:initializers.obj
 0002:000001ac       ___xi_a                    100081ac     MSVCRT:initializers.obj
 0002:000001b0       ___xi_z                    100081b0     MSVCRT:initializers.obj
 0002:000001b4       ___xp_a                    100081b4     MSVCRT:initializers.obj
 0002:000001b8       ___xp_z                    100081b8     MSVCRT:initializers.obj
 0002:000001bc       ___xt_a                    100081bc     MSVCRT:initializers.obj
 0002:000001c0       ___xt_z                    100081c0     MSVCRT:initializers.obj
 0002:000001d0       ??_C@_0BN@PPKEDFNA@?$CILjava?1util?1Vector?$DLIIIFIZZ?$CJV@ 100081d0     DirectAudioDevice.obj
 0002:000001f0       ??_C@_09OBBPPKHG@addFormat@ 100081f0     DirectAudioDevice.obj
 0002:000001fc       __real@3f800000            100081fc     DirectAudioDevice.obj
 0002:00000200       __real@3f847ae147ae147b    10008200     DirectAudioDevice.obj
 0002:00000210       __xmm@7fffffff7fffffff7fffffff7fffffff 10008210     DirectAudioDevice.obj
 0002:00000220       ??_C@_0N@FMCAPCBL@Unknown?5Name@ 10008220     DirectAudioDeviceProvider.obj
 0002:00000230       ??_C@_0P@JELLBOOJ@Unknown?5Vendor@ 10008230     DirectAudioDeviceProvider.obj
 0002:00000240       ??_C@_0BE@GEPKBKKC@Unknown?5Description@ 10008240     DirectAudioDeviceProvider.obj
 0002:00000254       ??_C@_0BA@LFHNEBGG@Unknown?5Version@ 10008254     DirectAudioDeviceProvider.obj
 0002:00000268       ??_C@_0EE@IPKJIHIL@com?1sun?1media?1sound?1DirectAudio@ 10008268     DirectAudioDeviceProvider.obj
 0002:000002b0       ??_C@_0EP@IBGEIIFD@?$CIIIILjava?1lang?1String?$DLLjava?1lan@ 100082b0     DirectAudioDeviceProvider.obj
 0002:00000300       ??_C@_06FALKBLGB@?$DMinit?$DO@ 10008300     DirectAudioDeviceProvider.obj
 0002:00000308       ??_C@_0CK@BNIEGIBB@javax?1sound?1midi?1MidiUnavailabl@ 10008308     MidiInDevice.obj
 0002:00000334       ??_C@_05NPPFNMNL@?$CIIJ?$CJV@ 10008334     MidiInDevice.obj
 0002:0000033c       ??_C@_0BF@LEBFAHIB@callbackShortMessage@ 1000833c     MidiInDevice.obj
 0002:00000354       ??_C@_06PFGPJLID@?$CI?$FLBJ?$CJV@ 10008354     MidiInDevice.obj
 0002:0000035c       ??_C@_0BE@CLHHHCK@callbackLongMessage@ 1000835c     MidiInDevice.obj
 0002:00000370       ??_C@_0N@JNOBNNBP@Unknown?5name@ 10008370     MidiInDeviceProvider.obj
 0002:00000380       ??_C@_0P@FLAGCHHF@Unknown?5vendor@ 10008380     MidiInDeviceProvider.obj
 0002:00000390       ??_C@_0BF@LIAFPILD@No?5details?5available@ 10008390     MidiInDeviceProvider.obj
 0002:000003a8       ??_C@_0BA@EMALCDDA@Unknown?5version@ 100083a8     MidiInDeviceProvider.obj
 0002:000003b8       ??_C@_0BF@HPHHCMEI@DirectSound?5Playback@ 100083b8     PLATFORM_API_WinOS_DirectSound.obj
 0002:000003d0       ??_C@_0BE@OBEMNMJC@DirectSound?5Capture@ 100083d0     PLATFORM_API_WinOS_DirectSound.obj
 0002:000003e4       ??_C@_05KBEOJPB@?$CFd?4?$CFd@ 100083e4     PLATFORM_API_WinOS_MidiIn.obj
 0002:000003ec       ??_C@_0BD@GIDICAOP@External?5MIDI?5Port@ 100083ec     PLATFORM_API_WinOS_MidiOut.obj
 0002:00000400       ??_C@_0CB@BKPHBOPD@Internal?5square?5wave?5synthesize@ 10008400     PLATFORM_API_WinOS_MidiOut.obj
 0002:00000424       ??_C@_0BI@BENILECD@Internal?5FM?5synthesizer@ 10008424     PLATFORM_API_WinOS_MidiOut.obj
 0002:0000043c       ??_C@_0BP@HFJPHHGA@Internal?5synthesizer?5?$CIgeneric?$CJ@ 1000843c     PLATFORM_API_WinOS_MidiOut.obj
 0002:0000045c       ??_C@_0BE@GKHJJDH@Windows?5MIDI_MAPPER@ 1000845c     PLATFORM_API_WinOS_MidiOut.obj
 0002:00000470       ??_C@_0BO@JHOFOEDM@Internal?5software?5synthesizer@ 10008470     PLATFORM_API_WinOS_MidiOut.obj
 0002:00000490       ??_C@_0L@CPKCBHCN@Port?5Mixer@ 10008490     PLATFORM_API_WinOS_Ports.obj
 0002:0000049b       ??_C@_00CNPNBAHC@@         1000849b     PLATFORM_API_WinOS_Ports.obj
 0002:0000049c       __real@3f000000            1000849c     PLATFORM_API_WinOS_Ports.obj
 0002:000004a0       __real@40000000            100084a0     PLATFORM_API_WinOS_Ports.obj
 0002:000004a4       __real@bf800000            100084a4     PLATFORM_API_WinOS_Ports.obj
 0002:000004b0       __xmm@41f00000000000000000000000000000 100084b0     PLATFORM_API_WinOS_Ports.obj
 0002:000004c0       ??_C@_0BG@PNPJGPKL@feature?5not?5supported@ 100084c0     PlatformMidi.obj
 0002:000004d8       ??_C@_0BC@GOGOPKAK@invalid?5device?5ID@ 100084d8     PlatformMidi.obj
 0002:000004ec       ??_C@_0BP@CMLKCPDD@internal?5error?3?5invalid?5handle@ 100084ec     PlatformMidi.obj
 0002:0000050c       ??_C@_0O@BNNCBLEN@out?5of?5memory@ 1000850c     PlatformMidi.obj
 0002:0000051c       ??_C@_0CH@PANCBAOC@com?1sun?1media?1sound?1PortMixer$B@ 1000851c     PortMixer.obj
 0002:00000544       ??_C@_0BH@DOGHFNPN@?$CIJLjava?1lang?1String?$DL?$CJV@ 10008544     PortMixer.obj
 0002:0000055c       ??_C@_04IOCNJLNK@Mute@     1000855c     PortMixer.obj
 0002:00000564       ??_C@_06HJGPBJLE@Select@   10008564     PortMixer.obj
 0002:0000056c       ??_C@_0CH@ECCNHGI@com?1sun?1media?1sound?1PortMixer$C@ 1000856c     PortMixer.obj
 0002:00000594       ??_C@_0DE@OMOINGJL@?$CILjava?1lang?1String?$DL?$FLLjavax?1soun@ 10008594     PortMixer.obj
 0002:000005c8       ??_C@_0BM@GDMEENBL@javax?1sound?1sampled?1Control@ 100085c8     PortMixer.obj
 0002:000005e4       ??_C@_0CI@OPKAAKLF@com?1sun?1media?1sound?1PortMixer$F@ 100085e4     PortMixer.obj
 0002:0000060c       ??_C@_0CM@PEFBHGMP@?$CIJLjava?1lang?1String?$DLFFFLjava?1la@ 1000860c     PortMixer.obj
 0002:00000638       ??_C@_0BL@HJNALIL@?$CIJIFFFLjava?1lang?1String?$DL?$CJV@ 10008638     PortMixer.obj
 0002:00000654       ??_C@_0BG@JLFLBLJI@?$CILjava?1lang?1Object?$DL?$CJV@ 10008654     PortMixer.obj
 0002:0000066c       ??_C@_0L@MNLDOJKN@addElement@ 1000866c     PortMixer.obj
 0002:00000678       ??_C@_0DE@HOKEHCEP@com?1sun?1media?1sound?1PortMixerPr@ 10008678     PortMixerProvider.obj
 0002:000006b0       ??_C@_0EN@JGCFGEEO@?$CIILjava?1lang?1String?$DLLjava?1lang?1@ 100086b0     PortMixerProvider.obj
 0002:00000784       __pRawDllMain              10008784     MSVCRT:dll_dllmain.obj
 0002:00000784       __pDefaultRawDllMain       10008784     MSVCRT:dll_dllmain.obj
 0002:00000794       ??_7exception@std@@6B@     10008794     MSVCRT:throw_bad_alloc.obj
 0002:0000079c       ??_C@_0BC@EOODALEL@Unknown?5exception@ 1000879c     MSVCRT:throw_bad_alloc.obj
 0002:000007b4       ??_7bad_alloc@std@@6B@     100087b4     MSVCRT:throw_bad_alloc.obj
 0002:000007bc       ??_C@_0P@GHFPNOJB@bad?5allocation@ 100087bc     MSVCRT:throw_bad_alloc.obj
 0002:000007d0       ??_7bad_array_new_length@std@@6B@ 100087d0     MSVCRT:throw_bad_alloc.obj
 0002:000007d8       ??_C@_0BF@KINCDENJ@bad?5array?5new?5length@ 100087d8     MSVCRT:throw_bad_alloc.obj
 0002:000007f4       ??_7type_info@@6B@         100087f4     MSVCRT:std_type_info_static.obj
 0002:00000870       __load_config_used         10008870     MSVCRT:loadcfg.obj
 0002:00000910       ??_R4exception@std@@6B@    10008910     MSVCRT:throw_bad_alloc.obj
 0002:00000924       ??_R3exception@std@@8      10008924     MSVCRT:throw_bad_alloc.obj
 0002:00000934       ??_R2exception@std@@8      10008934     MSVCRT:throw_bad_alloc.obj
 0002:0000093c       ??_R1A@?0A@EA@exception@std@@8 1000893c     MSVCRT:throw_bad_alloc.obj
 0002:00000958       ??_R4bad_alloc@std@@6B@    10008958     MSVCRT:throw_bad_alloc.obj
 0002:0000096c       ??_R3bad_alloc@std@@8      1000896c     MSVCRT:throw_bad_alloc.obj
 0002:0000097c       ??_R2bad_alloc@std@@8      1000897c     MSVCRT:throw_bad_alloc.obj
 0002:00000988       ??_R1A@?0A@EA@bad_alloc@std@@8 10008988     MSVCRT:throw_bad_alloc.obj
 0002:000009a4       ??_R4bad_array_new_length@std@@6B@ 100089a4     MSVCRT:throw_bad_alloc.obj
 0002:000009b8       ??_R3bad_array_new_length@std@@8 100089b8     MSVCRT:throw_bad_alloc.obj
 0002:000009c8       ??_R2bad_array_new_length@std@@8 100089c8     MSVCRT:throw_bad_alloc.obj
 0002:000009d8       ??_R1A@?0A@EA@bad_array_new_length@std@@8 100089d8     MSVCRT:throw_bad_alloc.obj
 0002:000009f4       ??_R4type_info@@6B@        100089f4     MSVCRT:std_type_info_static.obj
 0002:00000a08       ??_R3type_info@@8          10008a08     MSVCRT:std_type_info_static.obj
 0002:00000a18       ??_R2type_info@@8          10008a18     MSVCRT:std_type_info_static.obj
 0002:00000a20       ??_R1A@?0A@EA@type_info@@8 10008a20     MSVCRT:std_type_info_static.obj
 0002:00000a40       ___safe_se_handler_table   10008a40     <linker-defined>
 0002:00000d28       ___rtc_iaa                 10008d28     MSVCRT:initsect.obj
 0002:00000d2c       ___rtc_izz                 10008d2c     MSVCRT:initsect.obj
 0002:00000d30       ___rtc_taa                 10008d30     MSVCRT:initsect.obj
 0002:00000d34       ___rtc_tzz                 10008d34     MSVCRT:initsect.obj
 0002:00000db4       __TI2?AVbad_alloc@std@@    10008db4     MSVCRT:throw_bad_alloc.obj
 0002:00000dc4       __CTA2?AVbad_alloc@std@@   10008dc4     MSVCRT:throw_bad_alloc.obj
 0002:00000dd0       __CT??_R0?AVbad_alloc@std@@@8??0bad_alloc@std@@QAE@ABV01@@Z12 10008dd0     MSVCRT:throw_bad_alloc.obj
 0002:00000dec       __CT??_R0?AVexception@std@@@8??0exception@std@@QAE@ABV01@@Z12 10008dec     MSVCRT:throw_bad_alloc.obj
 0002:00000e08       __TI3?AVbad_array_new_length@std@@ 10008e08     MSVCRT:throw_bad_alloc.obj
 0002:00000e18       __CTA3?AVbad_array_new_length@std@@ 10008e18     MSVCRT:throw_bad_alloc.obj
 0002:00000e28       __CT??_R0?AVbad_array_new_length@std@@@8??0bad_array_new_length@std@@QAE@ABV01@@Z12 10008e28     MSVCRT:throw_bad_alloc.obj
 0002:00001c04       __IMPORT_DESCRIPTOR_DSOUND 10009c04     dsound:DSOUND.dll
 0002:00001c18       __IMPORT_DESCRIPTOR_WINMM  10009c18     winmm:WINMM.dll
 0002:00001c2c       __IMPORT_DESCRIPTOR_USER32 10009c2c     user32:USER32.dll
 0002:00001c40       __IMPORT_DESCRIPTOR_ole32  10009c40     ole32:ole32.dll
 0002:00001c54       __IMPORT_DESCRIPTOR_KERNEL32 10009c54     kernel32:KERNEL32.dll
 0002:00001c68       __IMPORT_DESCRIPTOR_VCRUNTIME140 10009c68     vcruntime:VCRUNTIME140.dll
 0002:00001c7c       __IMPORT_DESCRIPTOR_api-ms-win-crt-heap-l1-1-0 10009c7c     ucrt:api-ms-win-crt-heap-l1-1-0.dll
 0002:00001c90       __IMPORT_DESCRIPTOR_api-ms-win-crt-string-l1-1-0 10009c90     ucrt:api-ms-win-crt-string-l1-1-0.dll
 0002:00001ca4       __IMPORT_DESCRIPTOR_api-ms-win-crt-stdio-l1-1-0 10009ca4     ucrt:api-ms-win-crt-stdio-l1-1-0.dll
 0002:00001cb8       __IMPORT_DESCRIPTOR_api-ms-win-crt-runtime-l1-1-0 10009cb8     ucrt:api-ms-win-crt-runtime-l1-1-0.dll
 0002:00001ccc       __IMPORT_DESCRIPTOR_api-ms-win-crt-math-l1-1-0 10009ccc     ucrt:api-ms-win-crt-math-l1-1-0.dll
 0002:00001ce0       __NULL_IMPORT_DESCRIPTOR   10009ce0     dsound:DSOUND.dll
 0003:00000014       __fltused                  1000b014     MSVCRT:fltused.obj
 0003:00000018       ___security_cookie_complement 1000b018     MSVCRT:gs_cookie.obj
 0003:0000001c       ___security_cookie         1000b01c     MSVCRT:gs_cookie.obj
 0003:00000020       ___scrt_native_dllmain_reason 1000b020     MSVCRT:utility.obj
 0003:00000030       ___isa_enabled             1000b030     MSVCRT:cpu_disp.obj
 0003:00000040       ___scrt_ucrt_dll_is_in_use 1000b040     MSVCRT:ucrt_stubs.obj
 0003:00000044       ??_R0?AVbad_alloc@std@@@8  1000b044     MSVCRT:throw_bad_alloc.obj
 0003:00000060       ??_R0?AVexception@std@@@8  1000b060     MSVCRT:throw_bad_alloc.obj
 0003:0000007c       ??_R0?AVbad_array_new_length@std@@@8 1000b07c     MSVCRT:throw_bad_alloc.obj
 0003:000000a4       ??_R0?AVtype_info@@@8      1000b0a4     MSVCRT:std_type_info_static.obj
 0003:000000c0       ?data@DS_StartBufferHelper@@1VData@1@A 1000b0c0     PLATFORM_API_WinOS_DirectSound.obj
 0003:00000890       ?_OptionsStorage@?1??__local_stdio_printf_options@@9@4_KA 1000b890     PLATFORM_API_WinOS_MidiIn.obj
 0003:00000898       ?data@MidiIn_OpenHelper@@1VData@1@A 1000b898     PLATFORM_API_WinOS_MidiIn.obj
 0003:00000a58       ___scrt_current_native_startup_state 1000ba58     MSVCRT:utility.obj
 0003:00000a5c       ___scrt_native_startup_lock 1000ba5c     MSVCRT:utility.obj
 0003:00000d9c       ___isa_available           1000bd9c     MSVCRT:cpu_disp.obj
 0003:00000da0       ___favor                   1000bda0     MSVCRT:cpu_disp.obj
 0003:00000da4       ___scrt_debugger_hook_flag 1000bda4     MSVCRT:utility_desktop.obj
 0003:00000da8       ?__type_info_root_node@@3U__type_info_node@@A 1000bda8     MSVCRT:tncleanup.obj
 0003:00000db0       ?_OptionsStorage@?1??__local_stdio_scanf_options@@9@4_KA 1000bdb0     MSVCRT:default_local_stdio_options.obj
 0003:00000db8       ___dyn_tls_init_callback   1000bdb8     <common>

 entry point at        0001:000062a4

 Static symbols

 0000:ffff2000       .debug$S                   10000000     kernel32:KERNEL32.dll
 0000:ffff2000       .debug$S                   10000000     kernel32:KERNEL32.dll
 0000:ffff2000       .debug$S                   10000000     kernel32:KERNEL32.dll
 0000:ffff2000       .debug$S                   10000000     kernel32:KERNEL32.dll
 0000:ffff2000       .debug$S                   10000000     dsound:DSOUND.dll
 0000:ffff2000       .debug$S                   10000000     dsound:DSOUND.dll
 0000:ffff2000       .debug$S                   10000000     dsound:DSOUND.dll
 0000:ffff2000       .debug$S                   10000000     dsound:DSOUND.dll
 0000:ffff2000       .debug$S                   10000000     dsound:DSOUND.dll
 0000:ffff2000       .debug$S                   10000000     dsound:DSOUND.dll
 0000:ffff2000       .debug$S                   10000000     winmm:WINMM.dll
 0000:ffff2000       .debug$S                   10000000     winmm:WINMM.dll
 0000:ffff2000       .debug$S                   10000000     winmm:WINMM.dll
 0000:ffff2000       .debug$S                   10000000     winmm:WINMM.dll
 0000:ffff2000       .debug$S                   10000000     winmm:WINMM.dll
 0000:ffff2000       .debug$S                   10000000     winmm:WINMM.dll
 0000:ffff2000       .debug$S                   10000000     winmm:WINMM.dll
 0000:ffff2000       .debug$S                   10000000     winmm:WINMM.dll
 0000:ffff2000       .debug$S                   10000000     winmm:WINMM.dll
 0000:ffff2000       .debug$S                   10000000     winmm:WINMM.dll
 0000:ffff2000       .debug$S                   10000000     winmm:WINMM.dll
 0000:ffff2000       .debug$S                   10000000     winmm:WINMM.dll
 0000:ffff2000       .debug$S                   10000000     winmm:WINMM.dll
 0000:ffff2000       .debug$S                   10000000     winmm:WINMM.dll
 0000:ffff2000       .debug$S                   10000000     winmm:WINMM.dll
 0000:ffff2000       .debug$S                   10000000     winmm:WINMM.dll
 0000:ffff2000       .debug$S                   10000000     winmm:WINMM.dll
 0000:ffff2000       .debug$S                   10000000     winmm:WINMM.dll
 0000:ffff2000       .debug$S                   10000000     winmm:WINMM.dll
 0000:ffff2000       .debug$S                   10000000     winmm:WINMM.dll
 0000:ffff2000       .debug$S                   10000000     winmm:WINMM.dll
 0000:ffff2000       .debug$S                   10000000     winmm:WINMM.dll
 0000:ffff2000       .debug$S                   10000000     winmm:WINMM.dll
 0000:ffff2000       .debug$S                   10000000     winmm:WINMM.dll
 0000:ffff2000       .debug$S                   10000000     winmm:WINMM.dll
 0000:ffff2000       .debug$S                   10000000     winmm:WINMM.dll
 0000:ffff2000       .debug$S                   10000000     winmm:WINMM.dll
 0000:ffff2000       .debug$S                   10000000     winmm:WINMM.dll
 0000:ffff2000       .debug$S                   10000000     winmm:WINMM.dll
 0000:ffff2000       .debug$S                   10000000     winmm:WINMM.dll
 0000:ffff2000       .debug$S                   10000000     winmm:WINMM.dll
 0000:ffff2000       .debug$S                   10000000     winmm:WINMM.dll
 0000:ffff2000       .debug$S                   10000000     user32:USER32.dll
 0000:ffff2000       .debug$S                   10000000     user32:USER32.dll
 0000:ffff2000       .debug$S                   10000000     ole32:ole32.dll
 0000:ffff2000       .debug$S                   10000000     ole32:ole32.dll
 0000:ffff2000       .debug$S                   10000000     ole32:ole32.dll
 0000:ffff2000       .debug$S                   10000000     kernel32:KERNEL32.dll
 0000:ffff2000       .debug$S                   10000000     kernel32:KERNEL32.dll
 0000:ffff2000       .debug$S                   10000000     kernel32:KERNEL32.dll
 0000:ffff2000       .debug$S                   10000000     kernel32:KERNEL32.dll
 0000:ffff2000       .debug$S                   10000000     kernel32:KERNEL32.dll
 0000:ffff2000       .debug$S                   10000000     kernel32:KERNEL32.dll
 0000:ffff2000       .debug$S                   10000000     kernel32:KERNEL32.dll
 0000:ffff2000       .debug$S                   10000000     kernel32:KERNEL32.dll
 0000:ffff2000       .debug$S                   10000000     kernel32:KERNEL32.dll
 0000:ffff2000       .debug$S                   10000000     jsound.exp
 0000:ffff2000       .debug$S                   10000000     kernel32:KERNEL32.dll
 0000:ffff2000       .debug$S                   10000000     kernel32:KERNEL32.dll
 0000:ffff2000       .debug$S                   10000000     kernel32:KERNEL32.dll
 0000:ffff2000       .debug$S                   10000000     kernel32:KERNEL32.dll
 0000:ffff2000       .debug$S                   10000000     kernel32:KERNEL32.dll
 0000:ffff2000       .debug$S                   10000000     kernel32:KERNEL32.dll
 0000:ffff2000       .debug$S                   10000000     ucrt:api-ms-win-crt-runtime-l1-1-0.dll
 0000:ffff2000       .debug$S                   10000000     ucrt:api-ms-win-crt-heap-l1-1-0.dll
 0000:ffff2000       .debug$S                   10000000     ucrt:api-ms-win-crt-runtime-l1-1-0.dll
 0000:ffff2000       .debug$S                   10000000     ucrt:api-ms-win-crt-runtime-l1-1-0.dll
 0000:ffff2000       .debug$S                   10000000     ucrt:api-ms-win-crt-math-l1-1-0.dll
 0000:ffff2000       .debug$S                   10000000     ucrt:api-ms-win-crt-runtime-l1-1-0.dll
 0000:ffff2000       .debug$S                   10000000     ucrt:api-ms-win-crt-runtime-l1-1-0.dll
 0000:ffff2000       .debug$S                   10000000     ucrt:api-ms-win-crt-runtime-l1-1-0.dll
 0000:ffff2000       .debug$S                   10000000     ucrt:api-ms-win-crt-runtime-l1-1-0.dll
 0000:ffff2000       .debug$S                   10000000     ucrt:api-ms-win-crt-runtime-l1-1-0.dll
 0000:ffff2000       .debug$S                   10000000     ucrt:api-ms-win-crt-runtime-l1-1-0.dll
 0000:ffff2000       .debug$S                   10000000     ucrt:api-ms-win-crt-runtime-l1-1-0.dll
 0000:ffff2000       .debug$S                   10000000     ucrt:api-ms-win-crt-runtime-l1-1-0.dll
 0000:ffff2000       .debug$S                   10000000     ucrt:api-ms-win-crt-runtime-l1-1-0.dll
 0000:ffff2000       .debug$S                   10000000     ucrt:api-ms-win-crt-stdio-l1-1-0.dll
 0000:ffff2000       .debug$S                   10000000     ucrt:api-ms-win-crt-string-l1-1-0.dll
 0000:ffff2000       .debug$S                   10000000     ucrt:api-ms-win-crt-string-l1-1-0.dll
 0000:ffff2000       .debug$S                   10000000     ucrt:api-ms-win-crt-heap-l1-1-0.dll
 0000:ffff2000       .debug$S                   10000000     ucrt:api-ms-win-crt-heap-l1-1-0.dll
 0000:ffff2000       .debug$S                   10000000     kernel32:KERNEL32.dll
 0000:ffff2000       .debug$S                   10000000     vcruntime:VCRUNTIME140.dll
 0000:ffff2000       .debug$S                   10000000     vcruntime:VCRUNTIME140.dll
 0000:ffff2000       .debug$S                   10000000     vcruntime:VCRUNTIME140.dll
 0000:ffff2000       .debug$S                   10000000     vcruntime:VCRUNTIME140.dll
 0000:ffff2000       .debug$S                   10000000     vcruntime:VCRUNTIME140.dll
 0000:ffff2000       .debug$S                   10000000     vcruntime:VCRUNTIME140.dll
 0000:ffff2000       .debug$S                   10000000     vcruntime:VCRUNTIME140.dll
 0000:ffff2000       .debug$S                   10000000     vcruntime:VCRUNTIME140.dll
 0000:ffff2000       .debug$S                   10000000     kernel32:KERNEL32.dll
 0000:ffff2000       .debug$S                   10000000     kernel32:KERNEL32.dll
 0000:ffff2000       .debug$S                   10000000     kernel32:KERNEL32.dll
 0000:ffff2000       .debug$S                   10000000     kernel32:KERNEL32.dll
 0000:ffff2000       .debug$S                   10000000     kernel32:KERNEL32.dll
 0001:00000000       ??__E?data@DS_StartBufferHelper@@1VData@1@A@@YAXXZ 10001000 f   PLATFORM_API_WinOS_DirectSound.obj
 0001:00000016       ??__E?data@MidiIn_OpenHelper@@1VData@1@A@@YAXXZ 10001016 f   PLATFORM_API_WinOS_MidiIn.obj
 0001:00000599       _MAP_ClipAndConvertToByte  10001599 f   DirectAudioDevice.obj
 0001:000005b5       _MAP_ClipAndConvertToShort 100015b5 f   DirectAudioDevice.obj
 0001:000005d0       _MAP_ClipAndConvertToShort_Swapped 100015d0 f   DirectAudioDevice.obj
 0001:00000601       _MAP_ClipAndConvertToUByte 10001601 f   DirectAudioDevice.obj
 0001:0000587b       ?find_pe_section@@YAPAU_IMAGE_SECTION_HEADER@@QAEI@Z 1000687b f   MSVCRT:utility.obj
 0001:00005bd0       $$000000                   10006bd0     MSVCRT:ftol3.obj
 0001:00005f50       $$000000                   10006f50     MSVCRT:llmul.obj
 0001:00005f84       ?dllmain_crt_dispatch@@YGHQAUHINSTANCE__@@KQAX@Z 10006f84 f   MSVCRT:dll_dllmain.obj
 0001:00005fd7       ?dllmain_crt_process_attach@@YAHQAUHINSTANCE__@@QAX@Z 10006fd7 f   MSVCRT:dll_dllmain.obj
 0001:000060e1       ?dllmain_crt_process_detach@@YAH_N@Z 100070e1 f   MSVCRT:dll_dllmain.obj
 0001:00006173       ?dllmain_dispatch@@YAHQAUHINSTANCE__@@KQAX@Z 10007173 f   MSVCRT:dll_dllmain.obj
 0001:00006279       ?dllmain_raw@@YGHQAUHINSTANCE__@@KQAX@Z 10007279 f   MSVCRT:dll_dllmain.obj
 0001:000066f0       $$000000                   100076f0     MSVCRT:sehprolg4.obj
 0001:0000676e       ___get_entropy             1000776e f   MSVCRT:gs_support.obj
 0001:00006a9c       ??__F?data@DS_StartBufferHelper@@1VData@1@A@@YAXXZ 10007a9c f   PLATFORM_API_WinOS_DirectSound.obj
 0001:00006aa6       ??__F?data@MidiIn_OpenHelper@@1VData@1@A@@YAXXZ 10007aa6 f   PLATFORM_API_WinOS_MidiIn.obj
 0002:000001a0       ??data$initializer$@DS_StartBufferHelper@@1P6AXXZA@@3P6AXXZA 100081a0     PLATFORM_API_WinOS_DirectSound.obj
 0002:000001a4       ??data$initializer$@MidiIn_OpenHelper@@1P6AXXZA@@3P6AXXZA 100081a4     PLATFORM_API_WinOS_MidiIn.obj
 0002:00000700       _Int32ToUInt32             10008700     MSVCRT:ftol3.obj
 0002:00000708       _DP2to32                   10008708     MSVCRT:ftol3.obj
 0002:00000710       _MantissaMask              10008710     MSVCRT:ftol3.obj
 0002:00000718       _IntegerBit                10008718     MSVCRT:ftol3.obj
 0002:00000720       _SignBit64                 10008720     MSVCRT:ftol3.obj
 0002:00000728       _MinFP64                   10008728     MSVCRT:ftol3.obj
 0002:00000730       _MinInt64                  10008730     MSVCRT:ftol3.obj
 0002:00000738       _MaxInt64                  10008738     MSVCRT:ftol3.obj
 0002:00000740       _MaxUInt64                 10008740     MSVCRT:ftol3.obj
 0002:00000748       _MaxFP32                   10008748     MSVCRT:ftol3.obj
 0002:00000750       _MinFP32                   10008750     MSVCRT:ftol3.obj
 0002:00000758       _MinSubInexact             10008758     MSVCRT:ftol3.obj
 0002:00000760       _FpExcptTable              10008760     MSVCRT:ftol3.obj
 0002:00000770       _i1075                     10008770     MSVCRT:ftol3.obj
 0002:00000774       _i1087                     10008774     MSVCRT:ftol3.obj
 0002:00000778       _x0800                     10008778     MSVCRT:ftol3.obj
 0002:0000077c       _x17FF                     1000877c     MSVCRT:ftol3.obj
 0002:00000780       _CWMask                    10008780     MSVCRT:ftol3.obj
 0002:00000788       _GS_ExceptionPointers      10008788     MSVCRT:gs_report.obj
 0002:00000d38       __sehtable$___scrt_is_nonwritable_in_current_image 10008d38     MSVCRT:utility.obj
 0002:00000d58       __sehtable$?dllmain_crt_process_attach@@YAHQAUHINSTANCE__@@QAX@Z 10008d58     MSVCRT:dll_dllmain.obj
 0002:00000d78       __sehtable$?dllmain_crt_process_detach@@YAH_N@Z 10008d78     MSVCRT:dll_dllmain.obj
 0002:00000d98       __sehtable$?dllmain_dispatch@@YAHQAUHINSTANCE__@@KQAX@Z 10008d98     MSVCRT:dll_dllmain.obj
 0002:00000e50       .edata                     10008e50     jsound.exp
 0002:00000e78       rgpv                       10008e78     jsound.exp
 0002:00000f44       rgszName                   10008f44     jsound.exp
 0002:00001010       rgwOrd                     10009010     jsound.exp
 0002:00001076       szName                     10009076     jsound.exp
 0002:00001081       $N00001                    10009081     jsound.exp
 0002:000010c6       $N00002                    100090c6     jsound.exp
 0002:00001117       $N00003                    10009117     jsound.exp
 0002:00001151       $N00004                    10009151     jsound.exp
 0002:00001187       $N00005                    10009187     jsound.exp
 0002:000011bd       $N00006                    100091bd     jsound.exp
 0002:000011fb       $N00007                    100091fb     jsound.exp
 0002:0000123b       $N00008                    1000923b     jsound.exp
 0002:00001276       $N00009                    10009276     jsound.exp
 0002:000012b6       $N00010                    100092b6     jsound.exp
 0002:000012eb       $N00011                    100092eb     jsound.exp
 0002:00001320       $N00012                    10009320     jsound.exp
 0002:00001362       $N00013                    10009362     jsound.exp
 0002:0000139a       $N00014                    1000939a     jsound.exp
 0002:000013da       $N00015                    100093da     jsound.exp
 0002:00001410       $N00016                    10009410     jsound.exp
 0002:00001445       $N00017                    10009445     jsound.exp
 0002:0000147b       $N00018                    1000947b     jsound.exp
 0002:000014bd       $N00019                    100094bd     jsound.exp
 0002:000014f8       $N00020                    100094f8     jsound.exp
 0002:00001538       $N00021                    10009538     jsound.exp
 0002:00001575       $N00022                    10009575     jsound.exp
 0002:000015b3       $N00023                    100095b3     jsound.exp
 0002:000015e4       $N00024                    100095e4     jsound.exp
 0002:0000161b       $N00025                    1000961b     jsound.exp
 0002:00001653       $N00026                    10009653     jsound.exp
 0002:00001683       $N00027                    10009683     jsound.exp
 0002:000016b4       $N00028                    100096b4     jsound.exp
 0002:000016e4       $N00029                    100096e4     jsound.exp
 0002:00001727       $N00030                    10009727     jsound.exp
 0002:00001763       $N00031                    10009763     jsound.exp
 0002:000017a4       $N00032                    100097a4     jsound.exp
 0002:000017e2       $N00033                    100097e2     jsound.exp
 0002:00001821       $N00034                    10009821     jsound.exp
 0002:00001853       $N00035                    10009853     jsound.exp
 0002:0000188c       $N00036                    1000988c     jsound.exp
 0002:000018bd       $N00037                    100098bd     jsound.exp
 0002:000018f9       $N00038                    100098f9     jsound.exp
 0002:00001936       $N00039                    10009936     jsound.exp
 0002:00001968       $N00040                    10009968     jsound.exp
 0002:000019a5       $N00041                    100099a5     jsound.exp
 0002:000019e6       $N00042                    100099e6     jsound.exp
 0002:00001a14       $N00043                    10009a14     jsound.exp
 0002:00001a51       $N00044                    10009a51     jsound.exp
 0002:00001a8c       $N00045                    10009a8c     jsound.exp
 0002:00001ac9       $N00046                    10009ac9     jsound.exp
 0002:00001b04       $N00047                    10009b04     jsound.exp
 0002:00001b38       $N00048                    10009b38     jsound.exp
 0002:00001b6d       $N00049                    10009b6d     jsound.exp
 0002:00001ba1       $N00050                    10009ba1     jsound.exp
 0002:00001bd5       $N00051                    10009bd5     jsound.exp
 0002:00001e8c       .idata$6                   10009e8c     dsound:DSOUND.dll
 0002:000020f2       .idata$6                   1000a0f2     winmm:WINMM.dll
 0002:00002126       .idata$6                   1000a126     user32:USER32.dll
 0002:00002166       .idata$6                   1000a166     ole32:ole32.dll
 0002:00002366       .idata$6                   1000a366     kernel32:KERNEL32.dll
 0002:00002414       .idata$6                   1000a414     vcruntime:VCRUNTIME140.dll
 0002:0000254e       .idata$6                   1000a54e     ucrt:api-ms-win-crt-heap-l1-1-0.dll
 0002:0000256e       .idata$6                   1000a56e     ucrt:api-ms-win-crt-string-l1-1-0.dll
 0002:00002590       .idata$6                   1000a590     ucrt:api-ms-win-crt-stdio-l1-1-0.dll
 0002:000025b0       .idata$6                   1000a5b0     ucrt:api-ms-win-crt-runtime-l1-1-0.dll
 0002:000025d2       .idata$6                   1000a5d2     ucrt:api-ms-win-crt-math-l1-1-0.dll
 0003:00000000       ?sampleRateArray@@3PAHA    1000b000     PLATFORM_API_WinOS_DirectSound.obj
 0003:00000004       ?channelsArray@@3PAHA      1000b004     PLATFORM_API_WinOS_DirectSound.obj
 0003:0000000c       ?bitsArray@@3PAHA          1000b00c     PLATFORM_API_WinOS_DirectSound.obj
 0003:000000ec       ?g_cacheCount@@3HA         1000b0ec     PLATFORM_API_WinOS_DirectSound.obj
 0003:000000f0       ?g_audioDeviceCache@@3PAUDS_AudioDeviceCache@@A 1000b0f0     PLATFORM_API_WinOS_DirectSound.obj
 0003:00000870       ?g_lastCacheRefreshTime@@3_KA 1000b870     PLATFORM_API_WinOS_DirectSound.obj
 0003:00000878       ?g_mixerCount@@3HA         1000b878     PLATFORM_API_WinOS_DirectSound.obj
 0003:0000087c       ?CLSID_DAUDIO_Zero@@3U_GUID@@A 1000b87c     PLATFORM_API_WinOS_DirectSound.obj
 0003:000008c8       ?winMidiInErrMsg@@3PADA    1000b8c8     PLATFORM_API_WinOS_MidiIn.obj
 0003:00000990       _winMidiOutErrMsg          1000b990     PLATFORM_API_WinOS_MidiOut.obj
 0003:00000a60       ?is_initialized_as_dll@@3_NA 1000ba60     MSVCRT:utility.obj
 0003:00000a61       ?module_local_atexit_table_initialized@@3_NA 1000ba61     MSVCRT:utility.obj
 0003:00000a64       ?module_local_atexit_table@@3U_onexit_table_t@@A 1000ba64     MSVCRT:utility.obj
 0003:00000a70       ?module_local_at_quick_exit_table@@3U_onexit_table_t@@A 1000ba70     MSVCRT:utility.obj
 0003:00000a7c       ?__proc_attached@@3HA      1000ba7c     MSVCRT:dll_dllmain.obj
 0003:00000a80       _GS_ExceptionRecord        1000ba80     MSVCRT:gs_report.obj
 0003:00000ad0       _GS_ContextRecord          1000bad0     MSVCRT:gs_report.obj
 0004:00000060       $R000000                   1000c060     jsound.dll.res
